******************************************************************************
               TMS320C6x Linker PC v7.4.2                      
******************************************************************************
>> Linked Wed Jul 31 15:02:57 2013

OUTPUT FILE NAME:   <Multicore_Navigator.out>
ENTRY POINT SYMBOL: "_c_int00"  address: 0c109560


MEMORY CONFIGURATION

         name            origin    length      used     unused   attr    fill
----------------------  --------  ---------  --------  --------  ----  --------
  VECTORS               00800000   00000200  00000000  00000200  RWIX
  LL2_RW_DATA           00800200   000bfe00  0006f6f0  00050710  RWIX
  SL2                   0c000000   00400000  0010c537  002f3ac9  RWIX
  DDR3_CODE             80000000   01000000  00000000  01000000  RWIX
  DDR3_R_DATA           81000000   01000000  00000000  01000000  RWIX
  DDR3_RW_DATA          82000000   0e000000  08480000  05b80000  RWIX


SEGMENT ALLOCATION MAP

run origin  load origin   length   init length attrs members
----------  ----------- ---------- ----------- ----- -------
00800200    00800200    0006c100   00000000    rw-
  00800200    00800200    0003c000   00000000    rw- PacketData.buffer_LL2
  0083c200    0083c200    00030100   00000000    rw- QMSS_Data.Descriptor_LL2
0086c300    0086c300    000021c0   000011c0    rw-
  0086c300    0086c300    000011c0   000011c0    rw- .far
  0086d4c0    0086d4c0    00001000   00000000    rw- .stack
0086e4c0    0086e4c0    00001340   00000a20    rw-
  0086e4c0    0086e4c0    00000a20   00000a20    rw- .fardata
  0086eee0    0086eee0    00000800   00000000    rw- .sysmem
  0086f6e0    0086f6e0    00000120   00000000    rw- .cio
0086f800    0086f800    000000f0   000000d8    rw-
  0086f800    0086f800    000000d8   000000d8    rw- .neardata
  0086f8d8    0086f8d8    00000018   00000000    rw- .bss
0c000000    0c000000    000fc200   00000000    rw-
  0c000000    0c000000    00080000   00000000    rw- PacketData.buffer_SL2
  0c080000    0c080000    00060200   00000000    rw- QMSS_Data.Descriptor_SL2
  0c0e0200    0c0e0200    0001c000   00000000    rw- QMSS_Data.linkingRAM1
0c0fc200    0c0fc200    0000fb1f   0000fb1f    r-x
  0c0fc200    0c0fc200    0000d940   0000d940    r-x .text
  0c109b40    0c109b40    000021df   000021df    r-- .const
0c10bd20    0c10bd20    00000818   00000818    r--
  0c10bd20    0c10bd20    00000818   00000818    r-- .cinit
82000000    82000000    08480000   00000000    rw-
  82000000    82000000    080c0000   00000000    rw- QMSS_Data.Descriptor_DDR
  8a0c0000    8a0c0000    003c0000   00000000    rw- PacketData.buffer_DDR


SECTION ALLOCATION MAP

 output                                  attributes/
section   page    origin      length       input sections
--------  ----  ----------  ----------   ----------------
PacketData.buffer_LL2 
*          0    00800200    0003c000     UNINITIALIZED
                  00800200    0003c000     MNav_Init.obj (PacketData.buffer_LL2)

QMSS_Data.Descriptor_LL2 
*          0    0083c200    00030100     UNINITIALIZED
                  0083c200    00030100     MNav_Init.obj (QMSS_Data.Descriptor_LL2)

.far       0    0086c300    000011c0     
                  0086c300    00001000     MNav_Test.obj (.far) [fill = 0]
                  0086d300    00000140     rts6600_elf.lib : defs.obj (.far) [fill = 0]
                  0086d440    00000068     K2_common.obj (.far) [fill = 0]
                  0086d4a8    00000010     K2_common.obj (.far:Core_MPAX)
                  0086d4b8    00000008     rts6600_elf.lib : trgdrv.obj (.far) [fill = 0]

.stack     0    0086d4c0    00001000     UNINITIALIZED
                  0086d4c0    00000008     rts6600_elf.lib : boot.obj (.stack)
                  0086d4c8    00000ff8     --HOLE--

.fardata   0    0086e4c0    00000a20     
                  0086e4c0    000002d0     MNav_Init.obj (.fardata:freeHostQueueCfgTable)
                  0086e790    000001e0     rts6600_elf.lib : defs.obj (.fardata:_ftable)
                  0086e970    00000150     MNav_Init.obj (.fardata:flowCfgTable)
                  0086eac0    000000a0     rts6600_elf.lib : lowlev.obj (.fardata:_stream)
                  0086eb60    00000090     MNav_Init.obj (.fardata:descMemRegionsCfg)
                  0086ebf0    00000078     rts6600_elf.lib : lowlev.obj (.fardata:_device)
                  0086ec68    00000070     MNav_Init.obj (.fardata:freeMonoQueueCfgTable)
                  0086ecd8    00000050     K2_common.obj (.fardata:gTimerRegs)
                  0086ed28    0000003c     K2_common.obj (.fardata:gMPU_Regs)
                  0086ed64    00000004     rts6600_elf.lib : defs.obj (.fardata)
                  0086ed68    00000038     K2_common.obj (.fardata:gEDMA_TC_Regs)
                  0086eda0    00000024     K2_common.obj (.fardata:internal_exception_str)
                  0086edc4    00000004     --HOLE--
                  0086edc8    00000020     K2_common.obj (.fardata:bus_err_stat_str)
                  0086ede8    00000020     K2_Navigator_init_drv.obj (.fardata:gQM_PDSP_Cmd)
                  0086ee08    00000020     K2_Navigator_init_drv.obj (.fardata:gQM_PDSP_CtrlRegs)
                  0086ee28    00000020     K2_Navigator_init_drv.obj (.fardata:gQM_PDSP_IRAM)
                  0086ee48    00000018     K2_common.obj (.fardata:Peri_MPU_err_type_str)
                  0086ee60    00000014     K2_common.obj (.fardata:gEDMA_CC_Regs)
                  0086ee74    0000000c     rts6600_elf.lib : exit.obj (.fardata)
                  0086ee80    0000000c                     : memory.obj (.fardata)
                  0086ee8c    00000004     --HOLE--
                  0086ee90    00000008     K2_common.obj (.fardata:Ns_str)
                  0086ee98    00000008     K2_Navigator_init_drv.obj (.fardata:gQM_CfgRegs)
                  0086eea0    00000008     K2_Navigator_init_drv.obj (.fardata:gQM_DMA_CfgRegs)
                  0086eea8    00000008     K2_Navigator_init_drv.obj (.fardata:gQM_DMA_RxChCfgRegs)
                  0086eeb0    00000008     K2_Navigator_init_drv.obj (.fardata:gQM_DMA_RxFlowCfgRegs)
                  0086eeb8    00000008     K2_Navigator_init_drv.obj (.fardata:gQM_DMA_TxChCfgRegs)
                  0086eec0    00000008     K2_Navigator_init_drv.obj (.fardata:gQM_DescriptorRegions)
                  0086eec8    00000008     K2_Navigator_init_drv.obj (.fardata:gQM_INTD_Regs)
                  0086eed0    00000008     K2_Navigator_init_drv.obj (.fardata:numLinkingEntry)
                  0086eed8    00000008     rts6600_elf.lib : _lock.obj (.fardata)

.sysmem    0    0086eee0    00000800     UNINITIALIZED
                  0086eee0    00000008     rts6600_elf.lib : memory.obj (.sysmem)
                  0086eee8    000007f8     --HOLE--

.cio       0    0086f6e0    00000120     UNINITIALIZED
                  0086f6e0    00000120     rts6600_elf.lib : trgmsg.obj (.cio)

.neardata 
*          0    0086f800    000000d8     
                  0086f800    0000009c     K2_common.obj (.neardata)
                  0086f89c    0000003c     K2_Navigator_init_drv.obj (.neardata)

.rodata    0    0086f8d8    00000000     UNINITIALIZED

.bss       0    0086f8d8    00000018     UNINITIALIZED
                  0086f8d8    00000010     MNav_Init.obj (.bss)
                  0086f8e8    00000008     MNav_Test.obj (.bss)

PacketData.buffer_SL2 
*          0    0c000000    00080000     UNINITIALIZED
                  0c000000    00080000     MNav_Init.obj (PacketData.buffer_SL2)

QMSS_Data.Descriptor_SL2 
*          0    0c080000    00060200     UNINITIALIZED
                  0c080000    00060200     MNav_Init.obj (QMSS_Data.Descriptor_SL2)

QMSS_Data.linkingRAM1 
*          0    0c0e0200    0001c000     UNINITIALIZED
                  0c0e0200    0001c000     MNav_Init.obj (QMSS_Data.linkingRAM1)

.text      0    0c0fc200    0000d940     
                  0c0fc200    00004460     K2_common.obj (.text)
                  0c100660    00001b60     K2_Navigator_init_drv.obj (.text)
                  0c1021c0    00000640     MNav_Init.obj (.text)
                  0c102800    00000600     K2_common.obj (.text:retain)
                  0c102e00    000005c0     rts6600_elf.lib : divd.obj (.text:__c6xabi_divd)
                  0c1033c0    000005c0                     : _printfi.obj (.text:_getarg_diouxp)
                  0c103980    00000460                     : _printfi.obj (.text:_printfi)
                  0c103de0    00000460                     : _printfi.obj (.text:_setfield)
                  0c104240    00000440     K2_common.obj (.text:Core_MPAX)
                  0c104680    000003a0     MNav_Test.obj (.text)
                  0c104a20    000003a0     rts6600_elf.lib : fputs.obj (.text:fputs)
                  0c104dc0    00000320                     : _printfi.obj (.text:_pproc_fge)
                  0c1050e0    000002e0                     : _printfi.obj (.text:_pproc_fwp)
                  0c1053c0    000002a0                     : _printfi.obj (.text:fcvt)
                  0c105660    00000280                     : divf.obj (.text:__c6xabi_divf)
                  0c1058e0    00000280                     : _printfi.obj (.text:ecvt)
                  0c105b60    00000280                     : memory.obj (.text:free)
                  0c105de0    00000240                     : imath64.obj (.text:__c6xabi_divull)
                  0c106020    00000240                     : _printfi.obj (.text:_pconv_e)
                  0c106260    00000240                     : _printfi.obj (.text:_pproc_diouxp)
                  0c1064a0    00000220                     : _printfi.obj (.text:_pproc_str)
                  0c1066c0    00000220                     : fputc.obj (.text:fputc)
                  0c1068e0    00000200                     : _printfi.obj (.text:_pconv_g)
                  0c106ae0    00000200                     : setvbuf.obj (.text:setvbuf)
                  0c106ce0    000001e0     MNav_Test_main.obj (.text)
                  0c106ec0    000001c0     rts6600_elf.lib : _printfi.obj (.text:_mcpy)
                  0c107080    000001a0                     : trgdrv.obj (.text:HOSTrename)
                  0c107220    000001a0                     : imath40.obj (.text:__c6xabi_divul)
                  0c1073c0    00000180                     : copy_decompress_rle.obj (.text:__TI_decompress_rle_core)
                  0c107540    00000180                     : memory.obj (.text:malloc)
                  0c1076c0    00000140                     : _printfi.obj (.text:_pproc_fflags)
                  0c107800    00000140                     : lowlev.obj (.text:getdevice)
                  0c107940    00000120                     : fclose.obj (.text:_closefile)
                  0c107a60    00000120                     : _printfi.obj (.text:_ltostr)
                  0c107b80    00000120                     : fseek.obj (.text:fseek)
                  0c107ca0    00000100                     : trgdrv.obj (.text:HOSTlseek)
                  0c107da0    00000100                     : autoinit.obj (.text:_auto_init_elf)
                  0c107ea0    00000100                     : _io_perm.obj (.text:_wrt_ok)
                  0c107fa0    00000100                     : cpy_tbl.obj (.text:copy_in)
                  0c1080a0    000000e0                     : trgdrv.obj (.text:HOSTopen)
                  0c108180    000000e0                     : _printfi.obj (.text:_div)
                  0c108260    000000e0                     : atoi.obj (.text:atoi)
                  0c108340    000000e0                     : lowlev.obj (.text:close)
                  0c108420    000000e0                     : copy_zero_init.obj (.text:decompress:ZI:__TI_zero_init)
                  0c108500    000000e0                     : ltoa.obj (.text:ltoa)
                  0c1085e0    000000e0                     : memset.obj (.text:memset)
                  0c1086c0    000000e0                     : printf.obj (.text:printf)
                  0c1087a0    000000c0                     : trgdrv.obj (.text:HOSTread)
                  0c108860    000000c0                     : trgdrv.obj (.text:HOSTunlink)
                  0c108920    000000c0                     : trgdrv.obj (.text:HOSTwrite)
                  0c1089e0    000000c0                     : divu.obj (.text:__divu)
                  0c108aa0    000000c0                     : fflush.obj (.text:_doflush)
                  0c108b60    000000c0                     : exit.obj (.text:exit)
                  0c108c20    000000c0                     : tls.obj (.text:tls:init:__TI_tls_init)
                  0c108ce0    000000a0                     : trgdrv.obj (.text:HOSTclose)
                  0c108d80    000000a0                     : fopen.obj (.text:_cleanup)
                  0c108e20    000000a0                     : _printfi.obj (.text:_ecpy)
                  0c108ec0    000000a0                     : _printfi.obj (.text:_fcpy)
                  0c108f60    000000a0                     : memory.obj (.text:_minit)
                  0c109000    000000a0                     : _printfi.obj (.text:_pconv_f)
                  0c1090a0    000000a0                     : lowlev.obj (.text:finddevice)
                  0c109140    000000a0                     : lowlev.obj (.text:lseek)
                  0c1091e0    000000a0                     : memcpy64.obj (.text:memcpy)
                  0c109280    000000a0                     : memory.obj (.text:minsert)
                  0c109320    000000a0                     : memory.obj (.text:mremove)
                  0c1093c0    000000a0                     : lowlev.obj (.text:write)
                  0c109460    00000080                     : fixfu.obj (.text:__c6xabi_fixfu)
                  0c1094e0    00000080                     : llshift.obj (.text:__c6xabi_llshl)
                  0c109560    00000080                     : boot.obj (.text:_c_int00)
                  0c1095e0    00000080                     : trgmsg.obj (.text:readmsg)
                  0c109660    00000080                     : lowlev.obj (.text:unlink)
                  0c1096e0    00000060                     : cpp_init.obj (.text:__TI_cpp_init)
                  0c109740    00000060                     : frcmpyd_div.obj (.text:__c6xabi_frcmpyd_div)
                  0c1097a0    00000060                     : llshift.obj (.text:__c6xabi_llshru)
                  0c109800    00000060                     : imath64.obj (.text:_subcull)
                  0c109860    00000060                     : memccpy.obj (.text:memccpy)
                  0c1098c0    00000060                     : trgmsg.obj (.text:writemsg)
                  0c109920    00000040                     : isinf.obj (.text:__c6xabi_isinf)
                  0c109960    00000040                     : _printfi.obj (.text:__c6xabi_isnan)
                  0c1099a0    00000040                     : strasg.obj (.text:__strasgi_64plus)
                  0c1099e0    00000040                     : args_main.obj (.text:_args_main)
                  0c109a20    00000040                     : fputs.obj (.text:puts)
                  0c109a60    00000020                     : negll.obj (.text:__c6xabi_negll)
                  0c109a80    00000020                     : _lock.obj (.text:_nop)
                  0c109aa0    00000020                     : printf.obj (.text:_outc)
                  0c109ac0    00000020                     : printf.obj (.text:_outs)
                  0c109ae0    00000020                     : exit.obj (.text:abort)
                  0c109b00    00000020                     : copy_decompress_none.obj (.text:decompress:none:__TI_decompress_none)
                  0c109b20    00000020                     : copy_decompress_rle.obj (.text:decompress:rle24:__TI_decompress_rle24)

.const     0    0c109b40    000021df     
                  0c109b40    00001740     K2_common.obj (.const:.string)
                  0c10b280    000006c4     MNav_Init.obj (.const:acc48_le)
                  0c10b944    00000154     K2_Navigator_init_drv.obj (.const:.string)
                  0c10ba98    00000101     rts6600_elf.lib : ctype.obj (.const:.string:_ctypes_)
                  0c10bb99    00000002                     : fputs.obj (.const:.string)
                  0c10bb9b    00000001     --HOLE-- [fill = 0]
                  0c10bb9c    0000009c     MNav_Test.obj (.const:.string)
                  0c10bc38    0000008c     MNav_Init.obj (.const:.string)
                  0c10bcc4    00000038     MNav_Test_main.obj (.const:.string)
                  0c10bcfc    00000023     rts6600_elf.lib : _printfi.obj (.const:.string)

.cinit     0    0c10bd20    00000818     
                  0c10bd20    0000067c     (.cinit..fardata.load) [load image, compression = rle]
                  0c10c39c    000000da     (.cinit..neardata.load) [load image, compression = rle]
                  0c10c476    00000002     --HOLE-- [fill = 0]
                  0c10c478    0000001a     (.cinit..far.load) [load image, compression = rle]
                  0c10c492    00000002     --HOLE-- [fill = 0]
                  0c10c494    0000000c     (__TI_handler_table)
                  0c10c4a0    00000008     (.cinit..bss.load) [load image, compression = zero_init]
                  0c10c4a8    00000008     (.cinit.PacketData.buffer_DDR.load) [load image, compression = zero_init]
                  0c10c4b0    00000008     (.cinit.PacketData.buffer_LL2.load) [load image, compression = zero_init]
                  0c10c4b8    00000008     (.cinit.PacketData.buffer_SL2.load) [load image, compression = zero_init]
                  0c10c4c0    00000008     (.cinit.QMSS_Data.Descriptor_DDR.load) [load image, compression = zero_init]
                  0c10c4c8    00000008     (.cinit.QMSS_Data.Descriptor_LL2.load) [load image, compression = zero_init]
                  0c10c4d0    00000008     (.cinit.QMSS_Data.Descriptor_SL2.load) [load image, compression = zero_init]
                  0c10c4d8    00000008     (.cinit.QMSS_Data.linkingRAM1.load) [load image, compression = zero_init]
                  0c10c4e0    00000058     (__TI_cinit_table)

QMSS_Data.Descriptor_DDR 
*          0    82000000    080c0000     UNINITIALIZED
                  82000000    080c0000     MNav_Init.obj (QMSS_Data.Descriptor_DDR)

PacketData.buffer_DDR 
*          0    8a0c0000    003c0000     UNINITIALIZED
                  8a0c0000    003c0000     MNav_Init.obj (PacketData.buffer_DDR)


LINKER GENERATED COPY TABLES

__TI_cinit_table @ 0c10c4e0 records: 11, size/record: 8, table size: 88
	.fardata: load addr=0c10bd20, load size=0000067c bytes, run addr=0086e4c0, run size=00000a20 bytes, compression=rle
	.neardata: load addr=0c10c39c, load size=000000da bytes, run addr=0086f800, run size=000000d8 bytes, compression=rle
	.far: load addr=0c10c478, load size=0000001a bytes, run addr=0086c300, run size=000011c0 bytes, compression=rle
	.bss: load addr=0c10c4a0, load size=00000008 bytes, run addr=0086f8d8, run size=00000018 bytes, compression=zero_init
	PacketData.buffer_DDR: load addr=0c10c4a8, load size=00000008 bytes, run addr=8a0c0000, run size=003c0000 bytes, compression=zero_init
	PacketData.buffer_LL2: load addr=0c10c4b0, load size=00000008 bytes, run addr=00800200, run size=0003c000 bytes, compression=zero_init
	PacketData.buffer_SL2: load addr=0c10c4b8, load size=00000008 bytes, run addr=0c000000, run size=00080000 bytes, compression=zero_init
	QMSS_Data.Descriptor_DDR: load addr=0c10c4c0, load size=00000008 bytes, run addr=82000000, run size=080c0000 bytes, compression=zero_init
	QMSS_Data.Descriptor_LL2: load addr=0c10c4c8, load size=00000008 bytes, run addr=0083c200, run size=00030100 bytes, compression=zero_init
	QMSS_Data.Descriptor_SL2: load addr=0c10c4d0, load size=00000008 bytes, run addr=0c080000, run size=00060200 bytes, compression=zero_init
	QMSS_Data.linkingRAM1: load addr=0c10c4d8, load size=00000008 bytes, run addr=0c0e0200, run size=0001c000 bytes, compression=zero_init


LINKER GENERATED HANDLER TABLE

__TI_handler_table @ 0c10c494 records: 3, size/record: 4, table size: 12
	index: 0, handler: __TI_decompress_rle24
	index: 1, handler: __TI_decompress_none
	index: 2, handler: __TI_zero_init


GLOBAL SYMBOLS: SORTED ALPHABETICALLY BY Name 

address    name
--------   ----
0c0ffbb8   Bus_error_handler
0c109ae0   C$$EXIT
0c109918   C$$IO$$
0c0fe224   EDMA_CC_error_handler
0c0fe434   EDMA_TC_error_handler
0c0fdf74   EDMA_copy
0c0fe560   EDMA_error_handler
0c0fd950   EDMA_init
0c0fdeb4   EDMA_wait
0c1001d4   EXC_NMI
0c100114   EXC_internal
0c1001ec   EXC_swgen
0c102800   Exception_service_routine
0c108ce0   HOSTclose
0c107ca0   HOSTlseek
0c1080a0   HOSTopen
0c1087a0   HOSTread
0c107080   HOSTrename
0c108860   HOSTunlink
0c108920   HOSTwrite
0c0fe188   IDMA_copy
0c0fe158   IDMA_wait
0c0fd130   K2_ARM_PLL_init
0c0fd1e0   K2_PASS_PLL_init
0c101170   KeyStone_Copy_FDQ
0c0fea44   KeyStone_CorePac_AID_map
0c0ffc94   KeyStone_EXC_external
0c0ff9ec   KeyStone_Exception_cfg
0c100d04   KeyStone_Host_Descriptor_Queues_init
0c1043d0   KeyStone_MPAX_seg_setup
0c0fed08   KeyStone_MSMC_MP_interrupt_en
0c0fee88   KeyStone_MSMC_protection_exception_handler
0c100fb0   KeyStone_Mono_Descriptor_Queues_init
0c0fcf4c   KeyStone_PLL_init
0c0feacc   KeyStone_PrivID_Remap
0c100930   KeyStone_QMSS_Descriptor_Regions_init
0c100828   KeyStone_QMSS_Linking_RAM_init
0c10140c   KeyStone_Qmss_Config_Acc_Channel
0c10176c   KeyStone_Qmss_Config_Reclaim_Queue
0c101230   KeyStone_Qmss_Download_Firmware
0c101700   KeyStone_Qmss_config_Acc_Timer
0c101630   KeyStone_Qmss_disable_Acc_Channel
0c0fec28   KeyStone_SES_MPAX_setup
0c0ff160   KeyStone_SL2_EDC_enable
0c0ff720   KeyStone_SL2_EDC_handler
0c0ff220   KeyStone_SL2_EDC_interrupt_en
0c0feb48   KeyStone_SMS_MPAX_setup
0c104574   KeyStone_XMC_MPAX_setup
0c0fd84c   KeyStone_disable_PSC_Power_Domain
0c0fd7f4   KeyStone_disable_PSC_module
0c0fd790   KeyStone_enable_PSC_module
0c0fcac0   KeyStone_main_PLL_init
0c0ff078   KeyStone_peripherals_MPU_excepiton_handler
0c0fef80   KeyStone_peripherals_MPU_fault_status
0c1017d4   KeyStone_pktDma_Global_Control
0c101860   KeyStone_pktDma_TxCh_config
0c1018b8   KeyStone_pktDma_configureRxFlow
0c100204   KeyStone_print_device_info
0c0fe794   L1D_memory_protection_cfg
0c0ff370   L1P_EDC_setup
0c0ff5f8   L1P_ED_handler
0c0fe704   L1P_memory_protection_cfg
0c0fe664   L1_MPPA_setup
0c0fe828   L1_cache_protection
0086f888   LL2_EDC_DMA_err_str
0086f88c   LL2_EDC_L1D_err_str
0086f890   LL2_EDC_L1P_err_str
0c0ff3f4   LL2_EDC_handler
0c0ff30c   LL2_EDC_scrub
0c0ff274   LL2_EDC_setup
0086f884   LL2_EDC_victim_err_str
0c0fe838   LL2_MPPA_setup
0c0fe8d4   LL2_Memory_Protection_cfg
0c100290   Memory_Address_Test
0c100514   Memory_Bus_Bit_Walking
0c1003d4   Memory_Fill_Test
0c102bac   Nested_Exception_service_routine
0086ee90   Ns_str
0c1024ac   PA_PktDMA_init
0086ee48   Peri_MPU_err_type_str
0c104870   PktDmaTest
0c102364   QMSS_PktDMA_init
0c102200   QMSS_init
0c0fd444   Reset_Timer
0c102448   SRIO_PktDMA_init
0c0fd74c   Service_Watchdog
0c0fd2d4   TSC_delay_ms
0c0fd38c   TSC_delay_us
0c0fd2c4   TSC_init
0c0fd490   Timer64_Init
0086f6e0   __CIOBUF_
0c10c4e0   __TI_CINIT_Base
0c10c538   __TI_CINIT_Limit
0c10c494   __TI_Handler_Table_Base
0c10c4a0   __TI_Handler_Table_Limit
UNDEFED    __TI_INITARRAY_Base
UNDEFED    __TI_INITARRAY_Limit
0086e4c0   __TI_STACK_END
00001000   __TI_STACK_SIZE
0086f800   __TI_STATIC_BASE
00000800   __TI_SYSMEM_SIZE
UNDEFED    __TI_TLS_INIT_Base
UNDEFED    __TI_TLS_INIT_Limit
00000001   __TI_args_main
0c1096e0   __TI_cpp_init
0c109b00   __TI_decompress_none
0c109b20   __TI_decompress_rle24
0086ee7c   __TI_enable_exit_profile_output
ffffffff   __TI_pprof_out_hndl
ffffffff   __TI_prof_data_size
ffffffff   __TI_prof_data_start
0c108c20   __TI_tls_init
0c108420   __TI_zero_init
ffffffff   __binit__
0c102e00   __c6xabi_divd
0c105660   __c6xabi_divf
0c1089e0   __c6xabi_divu
0c107220   __c6xabi_divul
0c105de0   __c6xabi_divull
0c109460   __c6xabi_fixfu
0c109740   __c6xabi_frcmpyd_div
0c109920   __c6xabi_isinf
0c1094e0   __c6xabi_llshl
0c1097a0   __c6xabi_llshru
0c109a60   __c6xabi_negll
0c1099a0   __c6xabi_strasgi_64plus
ffffffff   __c_args__
0c1089e0   __divu
0c1099a0   __strasgi_64plus
0c1099e0   _args_main
0c107da0   _auto_init_elf
0c109560   _c_int00
0c108d80   _cleanup
0086ee74   _cleanup_ptr
0c107940   _closefile
0c10ba98   _ctypes_
0c108aa0   _doflush
0086ee78   _dtors_ptr
0086ed64   _ft_end
0086e790   _ftable
0086eed8   _lock
0c108f60   _minit
0c109a80   _nop
0c103980   _printfi
0086d4c0   _stack
0c109800   _subcull
0086eee0   _sys_memory
0086d300   _tmpnams
0086eedc   _unlock
0c107ea0   _wrt_ok
0c109ae0   abort
0c10b280   acc48_le
0c108260   atoi
ffffffff   binit
0086f8ec   bufLen
0086edc8   bus_err_stat_str
0c0fd26c   calc_cycle_measure_overhead
0c102510   checkQueues
0c108340   close
0c107fa0   copy_in
0086f87c   cycle_measure_overhead
0086eb60   descMemRegionsCfg
0c0fd8fc   edma_TC_priority_cfg
0c0fd898   edma_channel_TC_cfg
0086d440   exception_record
0c108b60   exit
0086e970   flowCfgTable
0c1066c0   fputc
0c104a20   fputs
0c105b60   free
0086e4c0   freeHostQueueCfgTable
0086ec68   freeMonoQueueCfgTable
0c107b80   fseek
0086f874   gARM_Core_Speed_Hz
0086f808   gBootCfgRegs
0086f804   gCGEM_Regs
0086f81c   gCIC0_Regs
0086f820   gCIC1_Regs
0086f898   gCIC_EXC_out_num
0086f824   gCIC_Regs
0086f878   gDSP_Core_Speed_Hz
0086f828   gEDMA_CC0_Regs
0086f82c   gEDMA_CC1_Regs
0086f830   gEDMA_CC2_Regs
0086f834   gEDMA_CC3_Regs
0086f838   gEDMA_CC4_Regs
0086ee60   gEDMA_CC_Regs
0086f83c   gEDMA_TC_0_0_Regs
0086f840   gEDMA_TC_0_1_Regs
0086f844   gEDMA_TC_1_0_Regs
0086f848   gEDMA_TC_1_1_Regs
0086f84c   gEDMA_TC_1_2_Regs
0086f850   gEDMA_TC_1_3_Regs
0086f854   gEDMA_TC_2_0_Regs
0086f858   gEDMA_TC_2_1_Regs
0086f85c   gEDMA_TC_2_2_Regs
0086f860   gEDMA_TC_2_3_Regs
0086f864   gEDMA_TC_3_0_Regs
0086f868   gEDMA_TC_3_1_Regs
0086f86c   gEDMA_TC_4_0_Regs
0086f870   gEDMA_TC_4_1_Regs
0086ed68   gEDMA_TC_Regs
0086f818   gGPIO_Regs
0086ed28   gMPU_Regs
0086f814   gMSMC_Regs
0086f8c4   gNetCP_DMA_CfgRegs
0086f8cc   gNetCP_DMA_RxChCfgRegs
0086f8d4   gNetCP_DMA_RxFlowCfgRegs
0086f8c8   gNetCP_DMA_TxChCfgRegs
0086f8d0   gNetCP_DMA_TxChPriority
0086f80c   gPLLC_Regs
0086f810   gPSC_Regs
0086ee98   gQM_CfgRegs
0086eea0   gQM_DMA_CfgRegs
0086eea8   gQM_DMA_RxChCfgRegs
0086eeb0   gQM_DMA_RxFlowCfgRegs
0086eeb8   gQM_DMA_TxChCfgRegs
0086eec0   gQM_DescriptorRegions
0086eec8   gQM_INTD_Regs
0086ede8   gQM_PDSP_Cmd
0086ee08   gQM_PDSP_CtrlRegs
0086ee28   gQM_PDSP_IRAM
0086f8a0   gQueueManageProxyRegs
0086f89c   gQueueManageRegs
0086f8a4   gQueueManageVBUSM
0086f8a8   gQueueStatusConfigRegs
0086f8ac   gQueueThresholdStatus
0086f8b0   gSRIO_DMA_CfgRegs
0086f8b8   gSRIO_DMA_RxChCfgRegs
0086f8c0   gSRIO_DMA_RxFlowCfgRegs
0086f8b4   gSRIO_DMA_TxChCfgRegs
0086f8bc   gSRIO_DMA_TxChPriority
0086ecd8   gTimerRegs
0086f800   gXMC_Regs
0086f894   guwIntcCICExcEvtIdx
82000000   hostDescriptor_DDR
0083c200   hostDescriptor_LL2
0c080000   hostDescriptor_SL2
0086eda0   internal_exception_str
0c0e0200   linkingRAM1
0c104240   lock_mem_prot_regs
0c109140   lseek
0c108500   ltoa
0c106d90   main
0c107540   malloc
0086d4a8   mem_prot_key
0c109860   memccpy
0c1091e0   memcpy
0c0fed70   memory_protection_exception_handler
0c1085e0   memset
82080000   monoDescriptor_DDR
0084c200   monoDescriptor_LL2
0c0a0000   monoDescriptor_SL2
0086eed0   numLinkingEntry
8a0c0000   packetBuffer_DDR_Size0
8a100000   packetBuffer_DDR_Size1
8a180000   packetBuffer_DDR_Size2
8a280000   packetBuffer_DDR_Size3
00800200   packetBuffer_LL2_Size0
00804200   packetBuffer_LL2_Size1
0080c200   packetBuffer_LL2_Size2
0081c200   packetBuffer_LL2_Size3
0c000000   packetBuffer_SL2_Size0
0c020000   packetBuffer_SL2_Size1
0c040000   packetBuffer_SL2_Size2
0c060000   packetBuffer_SL2_Size3
0086f8e8   pktLen
0c1086c0   printf
0c109a20   puts
0c1095e0   readmsg
0c109660   remove
0c106ae0   setvbuf
0086f8dc   uiInitialHostFdqNum
0086f8e0   uiInitialMonoFdqNum
0086f880   uiLL2_scrub_addr
0086f8d8   uiUsedDescRegionNum
0086f8e4   uiUsedRxFlowNum
0086c300   uiaDescriptorBuffer
0c109660   unlink
0c104308   unlock_mem_prot_regs
0c1093c0   write
0c1098c0   writemsg


GLOBAL SYMBOLS: SORTED BY Symbol Address 

address    name
--------   ----
00000001   __TI_args_main
00000800   __TI_SYSMEM_SIZE
00001000   __TI_STACK_SIZE
00800200   packetBuffer_LL2_Size0
00804200   packetBuffer_LL2_Size1
0080c200   packetBuffer_LL2_Size2
0081c200   packetBuffer_LL2_Size3
0083c200   hostDescriptor_LL2
0084c200   monoDescriptor_LL2
0086c300   uiaDescriptorBuffer
0086d300   _tmpnams
0086d440   exception_record
0086d4a8   mem_prot_key
0086d4c0   _stack
0086e4c0   __TI_STACK_END
0086e4c0   freeHostQueueCfgTable
0086e790   _ftable
0086e970   flowCfgTable
0086eb60   descMemRegionsCfg
0086ec68   freeMonoQueueCfgTable
0086ecd8   gTimerRegs
0086ed28   gMPU_Regs
0086ed64   _ft_end
0086ed68   gEDMA_TC_Regs
0086eda0   internal_exception_str
0086edc8   bus_err_stat_str
0086ede8   gQM_PDSP_Cmd
0086ee08   gQM_PDSP_CtrlRegs
0086ee28   gQM_PDSP_IRAM
0086ee48   Peri_MPU_err_type_str
0086ee60   gEDMA_CC_Regs
0086ee74   _cleanup_ptr
0086ee78   _dtors_ptr
0086ee7c   __TI_enable_exit_profile_output
0086ee90   Ns_str
0086ee98   gQM_CfgRegs
0086eea0   gQM_DMA_CfgRegs
0086eea8   gQM_DMA_RxChCfgRegs
0086eeb0   gQM_DMA_RxFlowCfgRegs
0086eeb8   gQM_DMA_TxChCfgRegs
0086eec0   gQM_DescriptorRegions
0086eec8   gQM_INTD_Regs
0086eed0   numLinkingEntry
0086eed8   _lock
0086eedc   _unlock
0086eee0   _sys_memory
0086f6e0   __CIOBUF_
0086f800   __TI_STATIC_BASE
0086f800   gXMC_Regs
0086f804   gCGEM_Regs
0086f808   gBootCfgRegs
0086f80c   gPLLC_Regs
0086f810   gPSC_Regs
0086f814   gMSMC_Regs
0086f818   gGPIO_Regs
0086f81c   gCIC0_Regs
0086f820   gCIC1_Regs
0086f824   gCIC_Regs
0086f828   gEDMA_CC0_Regs
0086f82c   gEDMA_CC1_Regs
0086f830   gEDMA_CC2_Regs
0086f834   gEDMA_CC3_Regs
0086f838   gEDMA_CC4_Regs
0086f83c   gEDMA_TC_0_0_Regs
0086f840   gEDMA_TC_0_1_Regs
0086f844   gEDMA_TC_1_0_Regs
0086f848   gEDMA_TC_1_1_Regs
0086f84c   gEDMA_TC_1_2_Regs
0086f850   gEDMA_TC_1_3_Regs
0086f854   gEDMA_TC_2_0_Regs
0086f858   gEDMA_TC_2_1_Regs
0086f85c   gEDMA_TC_2_2_Regs
0086f860   gEDMA_TC_2_3_Regs
0086f864   gEDMA_TC_3_0_Regs
0086f868   gEDMA_TC_3_1_Regs
0086f86c   gEDMA_TC_4_0_Regs
0086f870   gEDMA_TC_4_1_Regs
0086f874   gARM_Core_Speed_Hz
0086f878   gDSP_Core_Speed_Hz
0086f87c   cycle_measure_overhead
0086f880   uiLL2_scrub_addr
0086f884   LL2_EDC_victim_err_str
0086f888   LL2_EDC_DMA_err_str
0086f88c   LL2_EDC_L1D_err_str
0086f890   LL2_EDC_L1P_err_str
0086f894   guwIntcCICExcEvtIdx
0086f898   gCIC_EXC_out_num
0086f89c   gQueueManageRegs
0086f8a0   gQueueManageProxyRegs
0086f8a4   gQueueManageVBUSM
0086f8a8   gQueueStatusConfigRegs
0086f8ac   gQueueThresholdStatus
0086f8b0   gSRIO_DMA_CfgRegs
0086f8b4   gSRIO_DMA_TxChCfgRegs
0086f8b8   gSRIO_DMA_RxChCfgRegs
0086f8bc   gSRIO_DMA_TxChPriority
0086f8c0   gSRIO_DMA_RxFlowCfgRegs
0086f8c4   gNetCP_DMA_CfgRegs
0086f8c8   gNetCP_DMA_TxChCfgRegs
0086f8cc   gNetCP_DMA_RxChCfgRegs
0086f8d0   gNetCP_DMA_TxChPriority
0086f8d4   gNetCP_DMA_RxFlowCfgRegs
0086f8d8   uiUsedDescRegionNum
0086f8dc   uiInitialHostFdqNum
0086f8e0   uiInitialMonoFdqNum
0086f8e4   uiUsedRxFlowNum
0086f8e8   pktLen
0086f8ec   bufLen
0c000000   packetBuffer_SL2_Size0
0c020000   packetBuffer_SL2_Size1
0c040000   packetBuffer_SL2_Size2
0c060000   packetBuffer_SL2_Size3
0c080000   hostDescriptor_SL2
0c0a0000   monoDescriptor_SL2
0c0e0200   linkingRAM1
0c0fcac0   KeyStone_main_PLL_init
0c0fcf4c   KeyStone_PLL_init
0c0fd130   K2_ARM_PLL_init
0c0fd1e0   K2_PASS_PLL_init
0c0fd26c   calc_cycle_measure_overhead
0c0fd2c4   TSC_init
0c0fd2d4   TSC_delay_ms
0c0fd38c   TSC_delay_us
0c0fd444   Reset_Timer
0c0fd490   Timer64_Init
0c0fd74c   Service_Watchdog
0c0fd790   KeyStone_enable_PSC_module
0c0fd7f4   KeyStone_disable_PSC_module
0c0fd84c   KeyStone_disable_PSC_Power_Domain
0c0fd898   edma_channel_TC_cfg
0c0fd8fc   edma_TC_priority_cfg
0c0fd950   EDMA_init
0c0fdeb4   EDMA_wait
0c0fdf74   EDMA_copy
0c0fe158   IDMA_wait
0c0fe188   IDMA_copy
0c0fe224   EDMA_CC_error_handler
0c0fe434   EDMA_TC_error_handler
0c0fe560   EDMA_error_handler
0c0fe664   L1_MPPA_setup
0c0fe704   L1P_memory_protection_cfg
0c0fe794   L1D_memory_protection_cfg
0c0fe828   L1_cache_protection
0c0fe838   LL2_MPPA_setup
0c0fe8d4   LL2_Memory_Protection_cfg
0c0fea44   KeyStone_CorePac_AID_map
0c0feacc   KeyStone_PrivID_Remap
0c0feb48   KeyStone_SMS_MPAX_setup
0c0fec28   KeyStone_SES_MPAX_setup
0c0fed08   KeyStone_MSMC_MP_interrupt_en
0c0fed70   memory_protection_exception_handler
0c0fee88   KeyStone_MSMC_protection_exception_handler
0c0fef80   KeyStone_peripherals_MPU_fault_status
0c0ff078   KeyStone_peripherals_MPU_excepiton_handler
0c0ff160   KeyStone_SL2_EDC_enable
0c0ff220   KeyStone_SL2_EDC_interrupt_en
0c0ff274   LL2_EDC_setup
0c0ff30c   LL2_EDC_scrub
0c0ff370   L1P_EDC_setup
0c0ff3f4   LL2_EDC_handler
0c0ff5f8   L1P_ED_handler
0c0ff720   KeyStone_SL2_EDC_handler
0c0ff9ec   KeyStone_Exception_cfg
0c0ffbb8   Bus_error_handler
0c0ffc94   KeyStone_EXC_external
0c100114   EXC_internal
0c1001d4   EXC_NMI
0c1001ec   EXC_swgen
0c100204   KeyStone_print_device_info
0c100290   Memory_Address_Test
0c1003d4   Memory_Fill_Test
0c100514   Memory_Bus_Bit_Walking
0c100828   KeyStone_QMSS_Linking_RAM_init
0c100930   KeyStone_QMSS_Descriptor_Regions_init
0c100d04   KeyStone_Host_Descriptor_Queues_init
0c100fb0   KeyStone_Mono_Descriptor_Queues_init
0c101170   KeyStone_Copy_FDQ
0c101230   KeyStone_Qmss_Download_Firmware
0c10140c   KeyStone_Qmss_Config_Acc_Channel
0c101630   KeyStone_Qmss_disable_Acc_Channel
0c101700   KeyStone_Qmss_config_Acc_Timer
0c10176c   KeyStone_Qmss_Config_Reclaim_Queue
0c1017d4   KeyStone_pktDma_Global_Control
0c101860   KeyStone_pktDma_TxCh_config
0c1018b8   KeyStone_pktDma_configureRxFlow
0c102200   QMSS_init
0c102364   QMSS_PktDMA_init
0c102448   SRIO_PktDMA_init
0c1024ac   PA_PktDMA_init
0c102510   checkQueues
0c102800   Exception_service_routine
0c102bac   Nested_Exception_service_routine
0c102e00   __c6xabi_divd
0c103980   _printfi
0c104240   lock_mem_prot_regs
0c104308   unlock_mem_prot_regs
0c1043d0   KeyStone_MPAX_seg_setup
0c104574   KeyStone_XMC_MPAX_setup
0c104870   PktDmaTest
0c104a20   fputs
0c105660   __c6xabi_divf
0c105b60   free
0c105de0   __c6xabi_divull
0c1066c0   fputc
0c106ae0   setvbuf
0c106d90   main
0c107080   HOSTrename
0c107220   __c6xabi_divul
0c107540   malloc
0c107940   _closefile
0c107b80   fseek
0c107ca0   HOSTlseek
0c107da0   _auto_init_elf
0c107ea0   _wrt_ok
0c107fa0   copy_in
0c1080a0   HOSTopen
0c108260   atoi
0c108340   close
0c108420   __TI_zero_init
0c108500   ltoa
0c1085e0   memset
0c1086c0   printf
0c1087a0   HOSTread
0c108860   HOSTunlink
0c108920   HOSTwrite
0c1089e0   __c6xabi_divu
0c1089e0   __divu
0c108aa0   _doflush
0c108b60   exit
0c108c20   __TI_tls_init
0c108ce0   HOSTclose
0c108d80   _cleanup
0c108f60   _minit
0c109140   lseek
0c1091e0   memcpy
0c1093c0   write
0c109460   __c6xabi_fixfu
0c1094e0   __c6xabi_llshl
0c109560   _c_int00
0c1095e0   readmsg
0c109660   remove
0c109660   unlink
0c1096e0   __TI_cpp_init
0c109740   __c6xabi_frcmpyd_div
0c1097a0   __c6xabi_llshru
0c109800   _subcull
0c109860   memccpy
0c1098c0   writemsg
0c109918   C$$IO$$
0c109920   __c6xabi_isinf
0c1099a0   __c6xabi_strasgi_64plus
0c1099a0   __strasgi_64plus
0c1099e0   _args_main
0c109a20   puts
0c109a60   __c6xabi_negll
0c109a80   _nop
0c109ae0   C$$EXIT
0c109ae0   abort
0c109b00   __TI_decompress_none
0c109b20   __TI_decompress_rle24
0c10b280   acc48_le
0c10ba98   _ctypes_
0c10c494   __TI_Handler_Table_Base
0c10c4a0   __TI_Handler_Table_Limit
0c10c4e0   __TI_CINIT_Base
0c10c538   __TI_CINIT_Limit
82000000   hostDescriptor_DDR
82080000   monoDescriptor_DDR
8a0c0000   packetBuffer_DDR_Size0
8a100000   packetBuffer_DDR_Size1
8a180000   packetBuffer_DDR_Size2
8a280000   packetBuffer_DDR_Size3
ffffffff   __TI_pprof_out_hndl
ffffffff   __TI_prof_data_size
ffffffff   __TI_prof_data_start
ffffffff   __binit__
ffffffff   __c_args__
ffffffff   binit
UNDEFED    __TI_INITARRAY_Base
UNDEFED    __TI_INITARRAY_Limit
UNDEFED    __TI_TLS_INIT_Base
UNDEFED    __TI_TLS_INIT_Limit

[282 symbols]
